:1000000009C022C021C03AC01FC01EC01DC01CC0F4
:100010001BC01AC011241FBECFE9CDBF10E0A0E65F
:10002000B0E0EEE2F2E003C0C89531960D92A03642
:10003000B107D1F710E0A0E6B0E001C01D92A036F4
:10004000B107E1F774D0F2C0DBCF982F8823A9F075
:1000500088B5816088BD919592BF89B7826089BF5C
:1000600085B7877E85BF85B7806285BF889585B750
:100070008F7D85BF89B78D7F89BF08951F920F92AD
:100080000FB60F9211240F900FBE0F901F9018956E
:10009000379A369A3699FECF20E030E090E1369AD2
:1000A0003699FECF85B1280F311D9150C1F7379891
:1000B000329522952F7023273F702327822F99276F
:1000C0000895BC9A89E1C1DFBC980895B09B0AC02D
:1000D000B19B05C0B29909C083E090E0089582E029
:1000E00090E0089580E090E0089581E090E0089528
:1000F0001F93182FCDDF8F3880F4112319F480E07F
:1001000090E013C0812FA1DFC3DF90E08F3840F073
:1001100081E09827892F992708C081E090E005C0E9
:1001200091E081E09827892F99271F910895CF9218
:10013000DF92FF920F931F93CF93DF9385B78F7B4F
:1001400085BF87EE88BB83B7856083BF83E287B9AD
:1001500078948DE77ADFBADF082F21E0F22E90E065
:10016000C92E90E0D92E09C0823039F1833009F4CC
:1001700039C089E16ADFFF24012FA8DF182F813001
:1001800041F0813088F78DE7B3DF882391F799DF5D
:10019000F0CFC0E0D0E0BD2DAC2D34D0802D082FA5
:1001A00080E0A6DF882381F00A3939F08AE9AC2F94
:1001B000BD2F082E2FD00936E1F2FF20D1F28DE7B6
:1001C00097DF8823B1F6E3CFFF20A9F7093689F23C
:1001D0008EE38EDF882369F689E6AC2FBD2F082ECB
:1001E00019D0C7CF033009F4C4CF8EE32EDF6EDF02
:1001F000833009F0BECF80E07BDF882309F4B9CFDC
:1002000060DFB7CFE199FECFBFBBAEBBE09A1196DE
:100210000DB20895E199FECFBFBBAEBB0DBA1196EA
:0E0220000FB6F894E29AE19A0FBE0895FFCF50
:00000001FF
